:020000040000FA
:0A000000000000005FEF00F076D072
:08001800C9D09EA8FED7AD6E11
:100020001200EA680250120FE96E031CEF160D066B
:10003000E86A0E5A0CE302C0E9FF0350EF1A000011
:1000400000D000D00D06D8A00E06F9E2EF1A12007B
:10005000E836E836FC0B0109C212C009C216C050CE
:10006000F80B0309C06E640E15D8C282C2B2FED767
:10007000C4CF15F0C350146E1200106A0F6EFF0E3D
:100080000F26102200D0D8A01200030E0E6EE60E2E
:1000900002D8F5D70E6AFE0F0D6EE86A0E5AD8A088
:1000A000120000000D0600D0F8D70D6E0EBE02D86B
:1000B0000D5012000D1E0E1E0D4A0E2A1200006A6F
:1000C0004F0EAF6EB06A240EAC6E900EAB6E000198
:1000D0000F0EC16E070EB46E0FEE7EF0ED6AE950A2
:1000E000EA10FCE1EF6AC69A470E926EE00E936E3C
:1000F000C00E946EC5D0F2A409D0F2941A4A1B2AFD
:10010000D6CF18F0D7CF19F0817A11009EAA19D056
:10011000060EAB1412E1E2CF32F0E1CF31F0332A18
:1001200012EE7BF03350E126000EE222AECFE7FF65
:1001300032C0E2FF31C0E1FF1100AE50AE50AB98CB
:10014000AB8811003350345C14E0342AEACF0EF04F
:10015000E9CF0DF002EE7BF03450E926000EEA22E2
:10016000EF50306E0EC0EAFF0DC0E9FFD8801200DC
:1001700004D0E868306ED8A012001200336A346AE6
:100180009D8A9F8AF28EF28C12009D9A02EE7BF07D
:10019000010EF46EF36AF306000EF45AEE6AF450A0
:1001A000F310F9E1336A346A9D8A1200F29EC2CFDD
:1001B0007BF3C1CF7CF3C0CF7DF3C4CF7EF3C3CF3D
:1001C0007FF3E0CF80F30DC081F30EC082F311C046
:1001D00083F313C084F314C085F315C086F3F3CF03
:1001E00087F3D8CF88F3E8CF89F3F28E0001A1928C
:1001F000F80EB36E620EB26E000E2ADF556E15C099
:1002000056F053C015F052C014F0525014265350FB
:100210001522525014265350152255501424526E54
:1002200056501520536ED89053325232D8905332D4
:1002300052325330F36E5230576EF3325732F29ED1
:100240007BC3C2FF7CC3C1FF7DC3C0FF7EC3C4FFAD
:100250007FC3C3FF80C3E0FF81C30DF082C30EF0F4
:1002600083C311F084C313F085C314F086C315F063
:1002700087C3F3FF88C3D8FF89C3E8FFF28E10005D
:1002800094908B9094928B9294948B94949A8B8A62
:1002900094968B9694988B987A807A92939A8A9A6D
:1002A00093908A9093928A9293948A949298899840
:1002B00092968996516A400E506E800E586E6E6A04
:1002C0005F6A6C6A500E6B6E640E626E6F6E939A0C
:1002D0008A8A320ED2DE939A8A9A2A6A2C6800EEB3
:1002E0003AF0140EEE68E82EFDD70C0EC16EC08EEB
:1002F000000EAEDE526E15C053F0030EE82EFED790
:100300000000010EA5DE5B6E15C05CF0030EE82E4A
:10031000FED70000020E9CDE5D6E15C05EF0030E7F
:10032000E82EFED70000EAEC07F028DF2EDFCD6ACA
:10033000F294F28A870ED56EB16AA192A082B36A56
:10034000B26AD08EA292B10EB16E96EC08F0800E19
:10035000546E586E400E506E020E5A6EA70E596EB5
:10036000D6CF18F0D7CF19F0EDDE30C01CF0ED0E6F
:100370001C5C09E3FE0E1C5C03E34BEF04F003D0AE
:100380001D6A4BEF04F01CAE38D01D6A8C0E1C5C4D
:1003900005E11CC01DF01E681F682DD09C0E1C5C62
:1003A00005E11CC01DF02068216825D0AC0E1C5C46
:1003B00005E11CC01DF0226823681DD0BC0E1C5C2A
:1003C00005E11CC01DF02468256815D0CC0E1C5C0E
:1003D00004E11CC01DF026680ED0DC0E1C5C04E19C
:1003E0001CC01DF0276807D0EC0E1C5C04E11CC08B
:1003F0001DF0286829684BEF04F01D5204E14BEF13
:1004000004F04BEF04F08C0E1D5C2CE11E2803E180
:100410001CC01EF026D01CC01FF0340E1E5C0CE366
:100420005F0E1E5C09E21D50F8DD1E500DEC00F061
:100430001F500DEC00F014D0780E1E5C0DE37F0E03
:100440001E5C0AE28C0E0DEC00F01E500DEC00F06C
:10045000000E0DEC00F004D07F0E1E5C01E18998C7
:100460001E6819D29C0E1D5CD8A454D0202803E12C
:100470001CC020F04ED01CC021F0215225E1340ECA
:10048000205C0DE35F0E205C0AE21D500DEC00F0D5
:1004900020500DEC00F021500DEC00F014D0780E3F
:1004A000205C0DE37F0E205C0AE21D500DEC00F095
:1004B00020500DEC00F0000E0DEC00F004D07F0E8B
:1004C000205C01E1899824D0340E205C0DE35F0E9E
:1004D000205C0AE21D500DEC00F020500DEC00F005
:1004E00021500DEC00F014D0780E205C0DE37F0E4F
:1004F000205C0AE21D500DEC00F020500DEC00F0E5
:1005000021500DEC00F004D07F0E205C01E18988C1
:100510002068C1D1AC0E1D5C0BE1222803E11CC098
:1005200022F005D01CC023F0CEEC07F02268B3D136
:10053000BC0E1D5CD8A48CD1242803E11CC024F07F
:1005400086D11CC025F0010E245C0AE1BC0E0DEC26
:1005500000F0010E0DEC00F025500DEC00F076D10E
:10056000030E245C0DE3080E245C0AE2BC0E0DECC5
:1005700000F024500DEC00F025500DEC00F066D199
:100580000A0E245CD8A49ED025C04FF03D683C687C
:100590003B683A68416840683F683E684D684C680F
:1005A0004B684A686FC062F08B964F506902F3CF78
:1005B00076F0F4CF77F0786A4F506A02F3507726DE
:1005C000F4507822796A070ED890793278327732EF
:1005D0007632E82EF9D776506524606E7750662023
:1005E000616E6050655C6150665806E3080E6524D4
:1005F000606E000E6620616E6750605C68506158E6
:1006000006E3080E675C606E000E6858616E6FC08E
:1006100062F06350605C6450615827E28B9A7AB054
:1006200003D08B987A807A926B501824146E6C5099
:100630001920156E000E1A20166E000E1B20176E64
:1006400062501424056E000E1520066E000E162052
:10065000076E000E1720086E08C03DF007C03CF082
:1006600006C03BF005C03AF02BD06050635C61508F
:10067000645826E28B9A7AB203D08B887A827A9079
:100680006B501824146E6C501920156E000E1A2031
:10069000166E000E1B20176E62501424056E000E9D
:1006A0001520066E000E1620076E000E1720086E2D
:1006B00008C041F007C040F006C03FF005C03EF062
:1006C0004E80C4D00B0E245C26E125C050F0400EB5
:1006D0005024586E580E585C02E2580E586E970E11
:1006E000585C02E3960E586E2A8459501824056E01
:1006F0005A501920066E000E1A20076E000E1B209D
:10070000086E08C045F007C044F006C043F005C0BD
:1007100042F04E809BD00D0E245C10E1BC0E0DEC1F
:1007200000F024500DEC00F0070E2514156A146E2D
:100730000DEC00F015500DEC00F088D00F0E245C8D
:100740000DE3150E245C0AE2BC0E0DEC00F0245003
:100750000DEC00F025500DEC00F078D01F0E245C5D
:100760000AE1156AD8902530146E5F086B6E000E92
:1007700015546C6E6BD0200E245C06E1400E2524CF
:100780006F6E6FC062F062D0210E245C19E1710EB1
:10079000255C02E3700E256E25507F08146E000E56
:1007A000D8A0FF0F156E010E1424596E000E1520EF
:1007B0005A6E030ED89059365A36E82EFBD746D0DB
:1007C000420E245C18E1BC0E0DEC00F0420E0DEC64
:1007D00000F025500DEC00F0255204E15190D6ECCC
:1007E00007F008D0518094908B90D8905430506E80
:1007F00054C058F02BD0450E245C0AE1BC0E0DEC21
:1008000000F0450E0DEC00F025500DEC00F01ED070
:10081000640E245C0DE36D0E245C0AE2BC0E0DEC4C
:1008200000F024500DEC00F025500DEC00F00ED03F
:100830007B0E245C0BE1BC0E0DEC00F07B0E0DEC8E
:1008400000F025500DEC00F092988998246823D090
:10085000CC0E1D5C0CE1262808E11CC026F0CC0E55
:100860000DEC00F026500DEC00F0266814D0EC0ED4
:100870001D5C11E1282803E11CC028F00CD01CC02D
:1008800029F0EC0E0DEC00F028500DEC00F0295092
:100890000DEC00F028685850575C19E02AB416D0C7
:1008A0002A8459501824056E5A501920066E000EDD
:1008B0001A20076E000E1B20086E08C045F007C006
:1008C00044F006C043F005C042F04E8008D02AA490
:1008D00006D02A9445684468436842684E804EB00A
:1008E00093EC07F0050E2C5CD8B083EF07F0365080
:1008F000185C3750195838501A5839501B58D8A01E
:1009000082EF07F0398E2C52D8A4D4D05FA046D005
:100910007AB203D08B887A827A908A908B9A8B965F
:10092000080E6524606E000E6620616ED8906B34F0
:10093000146E6C34156E166A1636176AD890143613
:100940001536163614501824056E15501920066EEB
:1009500016501A20076E17501B20086E08C041F071
:1009600007C040F006C03FF005C03EF08B86634AEA
:10097000642A040E1824056E000E1920066E000E5F
:100980001A20076E000E1B20086E08C04DF007C02D
:100990004CF006C04BF005C04AF08AD06150645C50
:1009A00013E16050635C10E18A908B8A8B963D68FE
:1009B0003C683B683A68416840683F683E684D68FB
:1009C0004C684B684A6874D08B9A7AB003D08B9885
:1009D0007A807A92040E1824056E000E1920066E95
:1009E000000E1A20076E000E1B20086E08C04DF086
:1009F00007C04CF006C04BF005C04AF0716A706A3F
:100A0000625201E06206625219E16050635C0D6E51
:100A1000615064580E6E56EC00F0706E0EC071F0AE
:100A200071520AE170506F5C07E370506F5C706E3A
:100A3000000E7154716E02D0716A706A1BC017F09B
:100A40001AC016F019C015F018C014F06B50142617
:100A50006C501522000E1622172262501424146EB8
:100A6000000E1520156E000E1620166E000E1720B3
:100A7000176E70501424056E71501520066E000E0E
:100A80001620076E000E1720086E08C03DF007C044
:100A90003CF006C03BF005C03AF08B86635202E1A1
:100AA000645205E06306000E645A000101D0898893
:100AB00081EF07F0010E2C5CD8A4CBD05FA246D00A
:100AC0007AB003D08B987A807A928A928B9A080EA9
:100AD000675C606E000E6858616ED8906B34146E5F
:100AE0006C34156E166A1636176AD8901436153699
:100AF000163614501824056E15501920066E16501F
:100B00001A20076E17501B20086E08C03DF007C062
:100B10003CF006C03BF005C03AF0040E1824056E08
:100B2000000E1920066E000E1A20076E000E1B2004
:100B3000086E08C04DF007C04CF006C04BF005C071
:100B40004AF08B866306000E645A82D06150645C62
:100B500013E16050635C10E18A928B8A8B96416846
:100B600040683F683E683D683C683B683A684D684D
:100B70004C684B684A686CD08B9A7AB203D08B88E9
:100B80007A827A90040E1824056E000E1920066EE3
:100B9000000E1A20076E000E1B20086E08C04DF0D4
:100BA00007C04CF006C04BF005C04AF0716A706A8D
:100BB000625201E06206625219E16050635C0D6EA0
:100BC000615064580E6E56EC00F0706E0EC071F0FD
:100BD00071520AE170506F5C07E370506F5C706E89
:100BE000000E7154716E02D0716A706A1BC017F0EA
:100BF0001AC016F019C015F018C014F06B50142666
:100C00006C501522000E1622172262501424146E06
:100C1000000E1520156E000E1620166E000E172001
:100C2000176E70501424056E71501520066E000E5C
:100C30001620076E000E1720086E08C041F007C08E
:100C400040F006C03FF005C03EF08B86634A642A40
:100C500058D1020E2C5CD8A4EAD08B925750585C25
:100C600008E18B902A9445684468436842688A94F6
:100C7000DDD05750585CD8B06BD08B94040E18243C
:100C8000056E000E1920066E000E1A20076E000E6B
:100C90001B20086E08C049F007C048F006C047F0A6
:100CA00005C046F08B822A845850575C0D6E0E6A40
:100CB000D8A00E0656EC00F0056E0EC006F0595096
:100CC000055C5A5006582EE259501824146E5A509A
:100CD0001920156E000E1A20166E000E1B20176EBE
:100CE0005850575C0D6E0E6AD8A00E0656EC00F0F8
:100CF000096E0EC00AF00B6A0C6A0950145C056E8E
:100D00000A501558066E0B501658076E0C5017589F
:100D1000086E08C045F007C044F006C043F005C0A7
:100D200042F014D059501824056E5A501920066EFE
:100D3000000E1A20076E000E1B20086E08C045F03A
:100D400007C044F006C043F005C042F081746ED085
:100D50005850575CD8B06AD08B84040E1824056EA6
:100D6000000E1920066E000E1A20076E000E1B20C2
:100D7000086E08C049F007C048F006C047F005C03B
:100D800046F08B822A845850575C0D6E0E6AD8A0AC
:100D90000E0656EC00F0056E0EC006F05950055CCC
:100DA0005A5006582EE259501824146E5A501920E1
:100DB000156E000E1A20166E000E1B20176E58506E
:100DC000575C0D6E0E6AD8A00E0656EC00F0096E48
:100DD0000EC00AF00B6A0C6A0950145C056E0A50CA
:100DE0001558066E0B501658076E0C501758086EA3
:100DF00008C045F007C044F006C043F005C042F00B
:100E000014D059501824056E5A501920066E000E41
:100E10001A20076E000E1B20086E08C045F007C0A0
:100E200044F006C043F005C042F081746AD0030E5E
:100E30002C5C06E149684868476846688B9261D037
:100E4000040E2C5CD8A45DD08B964D684C684B6822
:100E50004A687AA029D0A092010E28EC00F05B6EBF
:100E600015C05CF0A082010E5C5C1DE303E1190E6D
:100E70005B5C19E35F8064C066F063C065F0695035
:100E80006524676E6A506620686E6550605C6650C7
:100E90006158000104E266C061F065C060F03D6821
:100EA0003C683B683A6801D05F907AA229D0A09252
:100EB000020E28EC00F05D6E15C05EF0A082010EFF
:100EC0005E5C1DE303E1190E5D5C19E35F8264C0A3
:100ED00068F063C067F06950675C656E6A50685877
:100EE000666E6050675C61506858000104E268C03B
:100EF00061F067C060F0416840683F683E6801D0BB
:100F00005F9211D80ED01BAC0CD01B6A1A6A196AFA
:100F1000186A2B6A2A6A00EE3AF0140EEE68E82E80
:100F2000FDD7B0EF01F02C68398E356A050E355CBF
:100F300033E2D8903534E96EEA6AEA36E936EA36C1
:100F40003A0EE926000EEA22EFCF05F0ECCF06F0CC
:100F5000ECCF07F0ECCF08F03650055C3750065860
:100F6000385007583950085815E2D8903534E96E92
:100F7000EA6AEA36E936EA363A0EE926000EEA224D
:100F8000EFCF36F0ECCF37F0ECCF38F0ECCF39F0D4
:100F900035C02CF0352ACAE34E90120022681200A8
:100FA0002668120028681200276812002A6A9490A6
:100FB0008B808B928B94949A8B8A8B96929889983B
:100FC000020E5A6EA70E596E6C6A500E6B6E400E72
:100FD000626E120089888B9A010E3DEC00F08B98AE
:100FE0007A807A92010E3DEC00F08B96010E3DEC7A
:100FF00000F0800E646E636A140E6D6E5F905FB0D9
:1010000023D0010E28EC00F05B6E15C05CF0010EE1
:101010005C5C05E303E1190E5B5C01E35F800001AA
:101020000E6A640E0D6E820E026E080E036E11ECD7
:1010300000F06D503DEC00F0030E6D5C01E36D06B9
:101040006306000E645ADBD76E8064C066F063C02E
:1010500065F05F908B887A907A825F92140E6D6E45
:10106000010E3DEC00F05FB222D0020E28EC00F041
:101070005D6E15C05EF0010E5E5C05E303E1190EC6
:101080005D5C01E35F8200010E6A640E0D6E820EEC
:10109000026E080E036E11EC00F06D503DEC00F096
:1010A000030E6D5C01E36D06634A642ADCD764C0FD
:1010B00068F063C067F06550675C696E6650685899
:1010C0006A6E6E828B987A807A92D8906A30156EAA
:1010D0006930146E6524606E15506620616E1A0EBC
:1010E0006D6E010E3DEC00F06350605C6450615821
:1010F00014E20E6A640E0D6E820E026E080E036E0E
:1011000011EC00F06D503DEC00F0030E6D5C01E35E
:101110006D066306000E645AE7D75F925F908B8A74
:1011200064C061F063C060F0899812007C687B68DD
:101130005C0E7E6E7A0E7D6E590E806F850E7F6E10
:10114000580E826F140E816F560E846FA90E836F36
:10115000550E866F430E856F530E886FE30E876FB3
:10116000520E8A6F890E896F510E8C6F350E8B6F00
:101170004F0E8E6FE60E8D6F4E0E906F9C0E8F6F22
:101180004D0E926F580E916F4C0E946F190E936F17
:101190004A0E966FDF0E956F490E986FAA0E976FE5
:1011A000480E9A6F7A0E996F470E9C6F4F0E9B6F89
:1011B000460E9E6F290E9D6F450EA06F080E9F6F05
:1011C000430EA26FEB0EA16F420EA46FD30EA36F5E
:1011D000410EA66FBF0EA56F400EA86FB00EA76F91
:1011E0003F0EAA6FA50EA96F3E0EAC6F9E0EAB6FA1
:1011F0003D0EAE6F9C0EAD6F3C0EB06F9E0EAF6F8E
:101200003B0EB26FA40EB16F3A0EB46FAE0EB36F59
:10121000390EB66FBC0EB56F380EB86FCE0EB76F05
:10122000370EBA6FE30EB96F360EBC6FFD0EBB6F93
:10123000360EBE6F1A0EBD6F350EC06F3B0EBF6F00
:10124000340EC26F5F0EC16F330EC46F870EC36F53
:10125000320EC66FB20EC56F310EC86FE10EC76F8A
:10126000310ECA6F140EC96F300ECC6F490ECB6FA2
:101270002F0ECE6F820ECD6F2E0ED06FBE0ECF6FA3
:101280002D0ED26FFD0ED16F2D0ED46F3F0ED36F8A
:101290002C0ED66F850ED56F2B0ED86FCD0ED76F57
:1012A0002B0EDA6F180ED96F2A0EDC6F670EDB6F0C
:1012B000290EDE6FB80EDD6F290EE06F0C0EDF6FAA
:1012C000280EE26F620EE16F270EE46FBC0EE36F33
:1012D000270EE66F180EE56F260EE86F760EE76FA5
:1012E000250EEA6FD80EE96F250EEC6F3C0EEB6F02
:1012F000240EEE6FA20EED6F240EF06F0B0EEF6F4B
:10130000230EF26F760EF16F220EF46FE40EF36F80
:10131000220EF66F540EF56F210EF86FC60EF76FA2
:10132000210EFA6F3B0EF96F200EFC6FB20EFB6FB1
:10133000200EFE6F2B0EFD6F1F0E0101006FA60E1B
:101340000001FF6F1F0E0101026F240E016F1E0EC0
:10135000046FA30E036F1E0E066F250E056F1D0E84
:10136000086FA90E076F1D0E0A6F2E0E096F1C0E57
:101370000C6FB60E0B6F1C0E0E6F3F0E0D6F1B0E1B
:10138000106FCB0E0F6F1B0E126F580E116F1A0ECF
:10139000146FE80E136F1A0E166F790E156F1A0E72
:1013A000186F0B0E176F190E1A6FA00E196F190E0A
:1013B0001C6F360E1B6F180E1E6FCE0E1D6F180E93
:1013C000206F680E1F6F180E226F030E216F170E0D
:1013D000246FA00E236F170E266F3F0E256F160E7B
:1013E000286FDF0E276F160E2A6F800E296F160EDC
:1013F0002C6F240E2B6F150E2E6FC80E2D6F150E31
:10140000306F6E0E2F6F150E326F160E316F140E79
:10141000346FBF0E336F140E366F690E356F140EB6
:10142000386F150E376F130E3A6FC20E396F130EE9
:101430003C6F710E3B6F130E3E6F210E3D6F120E0F
:10144000406FD20E3F6F120E426F840E416F120E2C
:10145000446F380E436F110E466FED0E456F110E3F
:10146000486FA30E476F110E4A6F5A0E496F110E47
:101470004C6F120E4B6F100E4E6FCC0E4D6F100E48
:10148000506F870E4F6F100E526F420E516F0F0E3E
:10149000546F5369566FBD0E556F0F0E586F7C0E0B
:1014A000576F0F0E5A6F3D0E596F0E0E5C6FFE0E8A
:1014B0005B6F0E0E5E6FC00E5D6F0E0E606F830E63
:1014C0005F6F0E0E626F470E616F0E0E646F0C0E33
:1014D000636F0D0E666FD20E656F0D0E686F990EFD
:1014E000676F0D0E6A6F610E696F0D0E6C6F2A0EBD
:1014F0006B6F0C0E6E6FF40E6D6F0C0E706FBE0E78
:101500006F6F0C0E726F8A0E716F0C0E746F560E29
:10151000736F0C0E766F230E756F0B0E786FF10ED6
:10152000776F0B0E7A6FC00E796F356A0001800EEF
:10153000355C24E200EE7BF0D8903534E926000ECD
:10154000EA22EECF09F0EFCF0AF00A30066E09303A
:10155000056E0632053206320532063205320F0EAE
:10156000061600EE7BF0D8903534E926000EEA220C
:1015700005C0EEFF06C0EFFF352AD8E301017C6904
:101580007B69A20E7E6FC30E7D6F9A0E806F460E32
:101590007F6F960E826F320E816F920E846F3A0EBD
:1015A000836F8E0E866F5D0E856F8A0E886F9A0E22
:1015B000876F860E8A6FF00E896F830E8C6F5F0EB9
:1015C0008B6F7F0E8E6FE70E8D6F7C0E906F850E8A
:1015D0008F6F790E926F3B0E916F760E946F070EA0
:1015E000936F720E966FE80E956F6F0E986FDF0E09
:1015F000976F6C0E9A6FEA0E996F6A0E9C6F0A0EC7
:101600009B6F670E9E6F3C0E9D6F640EA06F820EE7
:101610009F6F610EA26FDA0EA16F5F0EA46F440E72
:10162000A36F5C0EA66FBF0EA56F5A0EA86F4C0E6F
:10163000A76F570EAA6FE90EA96F550EAC6F960EE5
:10164000AB6F530EAE6FAD6F510EB06F200EAF6F1C
:101650004E0EB26FFB0EB16F4C0EB46FE50EB36F52
:101660004A0EB66FDC0EB56F480EB86FE20EB76F5C
:10167000460EBA6FF50EB96F450EBC6F150EBB6FF7
:10168000430EBE6F420EBD6F410EC06F7B0EBF6F2B
:101690003F0EC26FC00EC16F3E0EC46F100EC36FFF
:1016A0003C0EC66F6D0EC56F3A0EC86FD40EC76F75
:1016B000390ECA6F460EC96F370ECC6FC20ECB6F94
:1016C000360ECE6F490ECD6F340ED06FDA0ECF6F5F
:1016D000330ED26F740ED16F320ED46F180ED36FDB
:1016E000300ED66FC50ED56F2F0ED86F7B0ED76F0D
:1016F0002E0EDA6F3A0ED96F2D0EDC6F020EDB6FF5
:101700002B0EDE6FD10EDD6F2A0EE06FA90EDF6F9C
:10171000290EE26F880EE16F280EE46F6F0EE36F03
:10172000270EE66F5E0EE56F260EE86F530EE76F2D
:10173000250EEA6F500EE96F240EEC6F540EEB6F1E
:10174000230EEE6F5E0EED6F220EF06F6F0EEF6FD9
:10175000210EF26F860EF16F200EF46FA30EF36F61
:101760001F0EF66FC60EF56F1E0EF86FEF0EF76FB9
:101770001E0EFA6FF96F1D0EFC6F520EFB6F1C0EE2
:10178000FE6F8C0EFD6F1B0E0201006FCB0E010170
:10179000FF6F1B0E0201026F0F0E016F1A0E046F16
:1017A000580E036F190E066FA50E056F180E086F01
:1017B000F80E076F180E0A6F4F0E096F170E0C6F99
:1017C000AB0E0B6F170E0E6F0A0E0D6F160E106F0D
:1017D0006F0E0F6F150E126FD70E116F150E146F5F
:1017E000430E136F140E166FB30E156F140E186F91
:1017F000270E176F130E1A6F9F0E196F130E1C6FA3
:101800001A0E1B6F120E1E6F990E1D6F120E206F97
:101810001B0E1F6F110E226FA10E216F110E246F70
:10182000290E236F100E266FB50E256F100E286F30
:10183000440E276F0F0E2A6FD60E296F0F0E2C6FD6
:101840006B0E2B6F0F0E2E6F030E2D6F0E0E306F63
:101850009D0E2F6F0E0E326F3A0E316F0D0E346FDC
:10186000DA0E336F0D0E366F7C0E356F0D0E386F3E
:10187000210E376F0C0E3A6FC80E396F0C0E3C6F8D
:10188000720E3B6F0C0E3E6F1E0E3D6F0B0E406FC7
:10189000CC0E3F6F0B0E426F7C0E416F0B0E446FF0
:1018A0002E0E436F0A0E466FE30E456F0A0E486F09
:1018B000990E476F0A0E4A6F510E496F0A0E4C6F10
:1018C0000B0E4B6F090E4E6FC80E4D6F090E506F09
:1018D000850E4F6F090E526F450E516F090E546FF2
:1018E000060E536F080E566FC90E556F080E586FCF
:1018F0008E0E576F080E5A6F540E596F080E5C6F9C
:101900001C0E5B6F070E5E6FE50E5D6F070E606F5E
:10191000AF0E5F6F070E626F7B0E616F070E646F15
:10192000490E636F070E666F170E656F060E686FC0
:10193000E70E676F060E6A6FB90E696F060E6C6F61
:101940008B0E6B6F060E6E6F5F0E6D6F060E706FF7
:10195000340E6F6F060E726F0A0E716F050E746F84
:10196000E10E736F050E766FB90E756F050E786F09
:10197000930E776F050E7A6F6D0E796F000112006E
:02198000FFD78F
:020000040030CA
:0300010006170ED1
:020005008580F4
:060008000FC00FE00F40E5
:00000001FF
